S02000006F70656E626C745F6F6C696D65785F73746D3332703130332E7372656307
S3150800000000500020F14F0008395000083950000808
S31508000010395000083950000839500008000000001F
S315080000200000000000000000000000003950000831
S315080000303950000800000000395000084D07000834
S31508000040395000083950000839500008395000085E
S31508000050395000083950000839500008395000084E
S31508000060395000083950000839500008395000083E
S31508000070395000083950000839500008395000082E
S31508000080395000083950000839500008395000081E
S31508000090395000083950000839500008395000080E
S315080000A039500008395000083950000839500008FE
S315080000B039500008395000083950000839500008EE
S315080000C039500008395000083950000839500008DE
S315080000D039500008395000083950000839500008CE
S315080000E0395000083950000839500008000000004F
S315080000F000000000000000000000000000000000F2
S3110800010000000000000000005FF808F195
S3150800010C10B5054C237833B9044B13B10448AFF337
S3150800011C00800123237010BDE001002000000000C0
S3150800012CF050000808B5034B1BB103490348AFF35D
S3150800013C008008BD00000000E4010020F050000813
S3150800014C72B6704762B670472DE9F04184B0044622
S3150800015C0D4617469846684604F0E8F8164B029979
S3150800016CA3FB01318909002201E00132D2B2112A1E
S3150800017C1DD8124B13F8120003EB420393F801E057
S3150800018C00EB0E0303FB0443B1FBF3FC03FB1C1649
S3150800019C002EEAD11FFA8CF32B80013B9BB2B3F5E8
S315080001AC806FE2D2387088F800E0012000E0002069
S315080001BC04B0BDE8F08100BFD34D62103051000881
S315080001CC30B58DB00022ADF82E208DF82D200CAB55
S315080001DC03F8042D0DF12D020DF12E014FF4FA70D2
S315080001ECFFF7B2FF002837D01E4C1F4B23601F4B5E
S315080001FC23631F4B63630025A561E5612562656270
S3150800020CA562E562A560E5609DF82D30013B1B04EF
S3150800021C23619DF82C30013B1B056361BDF82E301C
S3150800022C6360204603F0ACFA0695079501230893FC
S3150800023C4CF6E042019202954FF6E07203920422C4
S3150800024C0492059509930E230A930DEB0201204699
S3150800025C03F012FA0DB030BDBA21064800F02AFB9D
S3150800026CC2E700BFFC0100200064004064020020C5
S3150800027C400200200851000810B50D4A136B40F2D5
S3150800028CE1741C60146B0023A360146BE360126B9F
S3150800029C116106E0064A126BC45C1A4414750133E4
S315080002ACDBB28B42F6D33221014803F00BFB10BDAF
S315080002BCFC01002038B504460D46002211461148AB
S315080002CC03F008FCD8B90F4B5B6B196840F26762F0
S315080002DC914203D0002098B1002309E09B68002BBB
S315080002ECF9D10120F7E71A44127DE2540133DBB247
S315080002FC044A526B11698B42F5D3297038BD00201C
S3150800030C38BD00BFFC01002008B5FFF719FF08BD72
S3150800031C10B500F0CDF900B910BD03F081F800282E
S3150800032CFAD000F065FB00F0D7F903F05DF900F0A0
S3150800033CC3F920F0604020F07F00044B986000F071
S3150800034CBBF94468FFF7FEFEA047E5E700ED00E0C1
S3150800035C70B508E0461C4D1C0B78037000F08EFB3C
S3150800036C304629462246531E9CB2002AF2D170BD4D
S3150800037C08B5C1F3080353B90368994209D040F884
S3150800038C041B4FF40072FFF7E3FF012008BD0020A1
S3150800039C08BD012008BD2DE9F041074603F084FD90
S315080003AC00247F2C14D83E68A30006EB03083B44B4
S315080003BC5D6800F063FB2A4600234146022003F0E1
S315080003CCCDFD38B956F824309D4209D10134E8E7F9
S315080003DC012400E0002403F081FD2046BDE8F081ED
S315080003EC0024F8E738B50D460B4B984208D004465E
S315080003FC0A4B994206D0FFF7CEFF20B9002407E036
S3150800040C074C00E0044C29462046FFF7B1FF08B11B
S3150800041C204638BD0024FBE7840400200060000851
S3150800042C800200202DE9F04106460C4617461D466B
S3150800043C21F4FF7828F001080368B3F1FF3F0DD0CB
S3150800044C3368984505D041463046FFF7CBFF06463C
S3150800045C28B33368E41A344404340CE04146FFF7F5
S3150800046C87FF03460028EBD116E017F8013B04F882
S3150800047C013B013D0FD000F001FB331DE31AB3F528
S3150800048C007FF2D308F500713046FFF7ABFF06463E
S3150800049C38B1041DE9E701231846BDE8F0810023AD
S315080004ACFAE70023F8E700004FF0FF33024A13601F
S315080004BC024A1360704700BF8002002084040020A3
S315080004CC10B54B1E114C241AA34218D8104B98423F
S315080004DC17D90B18013B0D4CA34214D80B460146F1
S315080004EC20F4FF7020F001000A4CA04203D00A4801
S315080004FCFFF798FF10BD0948FFF794FF10BD0020C1
S3150800050C10BD002010BD002010BD00BFFFFF010864
S3150800051CFF5F0008006000088002002084040020A9
S3150800052C30B587B0002305934A1E1F4B1B1A9A42F7
S3150800053C31D820F47F7323F003031C4A93422ED937
S3150800054C0A18013A184CA2422BD8C01A0144C1F316
S3150800055C8F25C1F3090109B10135ADB20024019407
S3150800056C03930123049303F09FFCA5420DD900F0D5
S3150800057C85FA05A901A803F063FD50B9039B03F599
S3150800058C806303930134A4B2EFE7012403F0A6FCBD
S3150800059C02E00024FAE70024204607B030BD002408
S315080005ACFAE70024F8E700BFFFFF0108FF5F000821
S315080005BC104B1B68B3F1FF3F1AD000B583B00D4A38
S315080005CC536891680B44D1680B4411690B44516903
S315080005DC0B4491690B44D26913445B4202AA42F854
S315080005EC043D04210448FFF76BFF03B05DF804FBD8
S315080005FC01207047840400200C6100080D4B1B6811
S3150800060C0D4A126813440D4A126813440C4A1268B0
S3150800061C13440C4A126813440B4A126813440B4AC7
S3150800062C126813440A4A1268D34201D00020704754
S3150800063C0120704700600008046000080860000884
S3150800064C0C600008106000081460000818600008A8
S3150800065C0C61000808B50C4B1B68B3F1FF3F04D0BE
S3150800066C0948FFF798FE034650B1084B1B68B3F1CF
S3150800067CFF3F07D00548FFF78EFE034600B101235E
S3150800068C184608BD0123FBE78404002080020020DD
S3150800069C004870470060000808B5FFF705FF08BD5D
S315080006AC08B5FFF70DFF08BD08B5FFF739FF08BDFC
S315080006BC08B5FFF7A3FF08BD08B5FFF7E9FF08BDA6
S315080006CC08B5FFF775FF034608B9184608BDFFF7C6
S315080006DCC1FF0346F9E700000022014B1A60704778
S315080006EC10E000E008B5FFF7F7FF054B054A5A601E
S315080006FC00229A6005211960034B1A6008BD00BFD9
S3150800070C10E000E03F19010088060020044B1B6826
S3150800071C13F4803F03D0034A136801331360704700
S3150800072C10E000E08806002008B5FFF7EFFF014B44
S3150800073C186808BD8806002008B5FFF7F5FF08BD40
S3150800074C70470000054B1B6813F0200F04D0034BB1
S3150800075C5B68037001207047002070470044004016
S3150800076C10B5094B5860FFF7DFFF00F10A04064B7A
S3150800077C1B6813F0800F05D100F080F9FFF7D4FF42
S3150800078C8442F4D210BD00BF0044004010B586B0B8
S3150800079C4FF46143009300230193029303930C22B5
S315080007AC04920593094C6946204603F0FFFD23691C
S315080007BC23F490432361636923F02A036361E36896
S315080007CC43F40053E36006B010BD00BF004400407C
S315080007DC70B506460D46402904D82846FFF7C0FFD3
S315080007EC00240BE06D21074800F064F8F5E700F0EB
S315080007FC45F9305DFFF7B4FF0134A4B2ABB29C42A5
S3150800080CF5D370BD5451000870B5254B1C78BCB98E
S3150800081C2448FFF797FF012801D0204670BD214BCD
S3150800082C1B78013BDBB23F2BF7D8FFF77DFF1E4B3E
S3150800083C186000221D4B1A700122194B1A70ECE72E
S3150800084C06460D46194B1B78013316481844FFF714
S3150800085C79FF044601280AD0FFF766FF124B1B687E
S3150800086C6433984219D900240D4B1C70D5E70F4BED
S3150800087C1A780132D2B21A700A4B1B789A4201D0F6
S3150800088C0024CAE70A493046FFF762FD0022044BEA
S3150800089C1A70064B1B782B70BFE70024BDE700BF08
S315080008ACCD0600208C060020D0060020CE0600209F
S315080008BC8D06002008B500F0E1F8FCE708B500F055
S315080008CCD5F8012806D000F067F918B10C4B1B783F
S315080008DC012B00D008BDFFF727FF0A4B1B680A4AF5
S315080008EC1268134403F5FA739842F3D30022044BA7
S315080008FC1A7000F05BF90028ECD1FFF709FDE9E75F
S3150800090CD8060020D4060020DC06002008B5054BC6
S3150800091C1B78012B00D008BDFFF706FF024B1860A9
S3150800092CF9E700BFD8060020DC06002008B501222E
S3150800093C034B1A70FFF7EAFFFFF7C0FF08BD00BFAD
S3150800094CD806002008B5FFF7DFFC00F093F8FFF790
S3150800095CC9FEFFF7A1FE00F007F900F00FF8FFF744
S3150800096CE5FF08BD08B500F089F8FFF7CFFE00F0E3
S3150800097C2BFA00F013F8FFF7A1FF08BD10B502F02B
S3150800098CBDFCFFF71DFC044C01232370FFF7FEFE8C
S3150800099C0023237010BD00BF0000002000B583B0F3
S315080009AC0DF107011048FFF785FC012809D00DF158
S315080009BC07010D48FFF728FF01280BD003B05DF897
S315080009CC04FB0122094B1A709DF80710064802F021
S315080009DCB5FCECE70022054B1A709DF80710024887
S315080009EC02F0ACFCEAE700BFE0060020000000209D
S315080009FC7047000038B504460D46094B1B78012B89
S31508000A0C05D0074B1B7833B102F090FC38BDC9B240
S31508000A1CFFF732FCF5E7E9B22046FFF7D9FEF3E714
S31508000A2C00000020074B1B78022B05D0032B05D0A2
S31508000A3C012B05D0402070470020704700207047D6
S31508000A4C0820704700000020074B1B78022B05D0A6
S31508000A5C032B05D0012B05D040207047002070478A
S31508000A6C00207047082070470000002008B502F0E7
S31508000A7C53FC08BD08B502F0E1FC08BD08B502F048
S31508000A8CE2FC08BD10B4034601310C4AA2FB032351
S31508000A9CDB08F9D100230B70084BA3FB0023DB08FA
S31508000AAC1A4603EB83035C00031B303301F8013D44
S31508000ABC1046002AF0D1084610BC7047CDCCCCCCD9
S31508000ACC00F00F03092802D903F13700704710B557
S31508000ADC03F1300404F0D0FA2044437803F00303FE
S31508000AEC022B01D0E0B210BD203CFBE738B5054619
S31508000AFC0C460009FFF7E4FF207005F00F00FFF71E
S31508000B0CDFFF60700023A370204638BDF8B5074692
S31508000B1C00252E4607E0203C10E03301DBB21344D7
S31508000B2CDEB20135EDB2012D19D87C5D04F0A4FABC
S31508000B3C2044437803F00303022BECD0E3B2A3F171
S31508000B4C3002D2B2162A09D8A3F13A01C9B206293B
S31508000B5C07D9092AE1D9373BDAB2DEE7002630464F
S31508000B6CF8BD0026FBE7000008B50022064B1A70F4
S31508000B7C0649074801F052FD00B908BD772105481A
S31508000B8CFFF798FEF9E700BF800B0020805100089C
S31508000B9C2807002084510008034B1B780BB1002052
S31508000BAC70470120704700BF800B002008B5FFF77F
S31508000BBC5DFF01280ED0084B1B780BB1002008BD31
S31508000BCC02F046FC012801D0002008BD0122024B88
S31508000BDC1A7008BD002008BD800B002038B50546E4
S31508000BEC047804F049FA2044437803F00303022BF3
S31508000BFC03D0532C03D0032038BD203CF9E704F06E
S31508000C0C3BFA6B781844427812F0040F01D1032092
S31508000C1C38BD312B07D0322B07D0332B01D003200C
S31508000C2C38BD022038BD002038BD012038BD70B54E
S31508000C3C06460230FFF76AFF054684B2043630468C
S31508000C4CFFF764FF0544EDB2013CA4B20236012C51
S31508000C5CF5D8ED43EDB23046FFF758FF854201D083
S31508000C6C002070BD012070BD2DE9F04104461646E2
S31508000C7C8846A1B198B12046FFF7B0FF0546032870
S31508000C8C00F099802046FFF7D2FF002800F09780E5
S31508000C9C012D2DD04DB1022D57D000278CE040F2F6
S31508000CAC61214848FFF706FEE5E7A01CFFF72EFF73
S31508000CBC87B2201DFFF72AFF0002C8F80000A01D06
S31508000CCCFFF724FFD8F800301844C8F80000083499
S31508000CDC033F3FB2002E6FD0002506E02046FFF7F3
S31508000CEC15FF705502340135ADB2BD42F6DB63E033
S31508000CFCA01CFFF70BFF87B2201DFFF707FF0004A8
S31508000D0CC8F80000A01DFFF701FFD8F8003003EB68
S31508000D1C0020C8F8000004F10800FFF7F7FED8F821
S31508000D2C00301844C8F800000A34043F3FB2002EBD
S31508000D3C42D0002506E02046FFF7E8FE705502343F
S31508000D4C0135ADB2BD42F6DB36E0A01CFFF7DEFE80
S31508000D5C87B2201DFFF7DAFE0006C8F80000A01DB2
S31508000D6CFFF7D4FED8F8003003EB0040C8F80000B3
S31508000D7C04F10800FFF7CAFED8F8003003EB002090
S31508000D8CC8F8000004F10A00FFF7C0FED8F80030D6
S31508000D9C1844C8F800000C34053F3FB266B100256C
S31508000DAC06E02046FFF7B2FE705502340135ADB2A7
S31508000DBCBD42F6DB00E000273846BDE8F0814FF06F
S31508000DCCFF37F9E784510008964B1B78002B00F087
S31508000DDCF18170B5012B05D0022B2DD0032B00F019
S31508000DEC3F8170BDFFF758FC02F054FB8E4802F0A9
S31508000DFC95FB8E4802F092FB02F048FB0122014655
S31508000E0C8B4801F037FC30B18A4802F087FB012089
S31508000E1C02F076FB70BD884802F080FB874802F02A
S31508000E2C7DFB874802F07AFB864B00221A605A60D3
S31508000E3C02227C4B1A7070BD834C04F50C724FF46D
S31508000E4C8071824802F030F894F84132002B5ED15A
S31508000E5C002877D07D48002200F5C071FFF704FF03
S31508000E6C0446B0F1FF3F60D0002C09DD754B5B687A
S31508000E7C002B69D1754BD3F88021724B1A605C60D4
S31508000E8C714BD3F84422D3F83C329A42A9D10021AB
S31508000E9C674801F0C5FE002840F0A980694B5B68DD
S31508000EAC73B3654802F03AFB694802F037FB694DA3
S31508000EBC644C29466068FFF7E5FD284602F02EFBD0
S31508000ECC654802F02BFB2946E078FFF70FFEA91CB4
S31508000EDCA078FFF70BFE291D6078FFF707FEA91D02
S31508000EEC2078FFF703FE284602F018FB5B4802F051
S31508000EFC15FB61682068FFF7D7FB002800F0848093
S31508000F0C4D4802F00BFB0322464B1A7070BD49483C
S31508000F1C02F004FB022002F0F3FA04F50C7001F05F
S31508000F2C6BFE00223F4B1A7070BD424802F0F6FA6F
S31508000F3C032002F0E5FA3E4801F05EFE0022394B2A
S31508000F4C1A7070BD00248FE7404AD2F880113D4ACA
S31508000F5C12681A44914239D0374802F0DFFA3C48F5
S31508000F6C02F0DCFA3B4E374D31466868FFF78AFDCE
S31508000F7C304602F0D3FA384802F0D0FA3146E8780F
S31508000F8CFFF7B4FDB11CA878FFF7B0FD311D6878E2
S31508000F9CFFF7ACFDB11D2878FFF7A8FD304602F027
S31508000FACBDFA2E4802F0BAFA69682868FFF77CFB86
S31508000FBC80B1214802F0B2FA214802F0AFFA234B6D
S31508000FCCD3F880211F4B1A605C6059E723441D4AED
S31508000FDC536055E7174802F0A1FA052002F090FA7B
S31508000FEC134801F009FE00220E4B1A7070BD114809
S31508000FFC02F094FA042002F083FA0D4801F0FCFD85
S3150800100C0022084B1A7070BD0A4802F087FA0520B0
S3150800101C02F076FA064801F0EFFD0022014B1A7031
S3150800102C70BD00BF800B0020A0510008C4510008F9
S3150800103C58090020EC510008F4510008FC5100082E
S3150800104C205200082007002028070020840B0020C7
S3150800105C50520008080D00205C5200080053000886
S3150800106C554C04F50C724FF48071544801F01CFF72
S3150800107C94F84132002B66D100287FD04F4800F5F2
S3150800108C807200F5C071FFF7EFFD0546B0F1FF3F22
S3150800109C67D0002D34DD4A4802F040FA494C214607
S315080010AC2846FFF7EFFC204602F038FA464802F0CD
S315080010BC35FA424E214696F88301FFF717FDA11C17
S315080010CC96F88201FFF712FD211D96F88101FFF7AC
S315080010DC0DFDA11D96F88001FFF708FD204602F0CC
S315080010EC1DFA3A4802F01AFA06F580722946D6F81D
S315080010FC8001FFF7D5FA002842D0354802F00EFADF
S3150800110C2D4BD3F84422D3F83C329A427FF469AE7D
S3150800111C304802F003FAFFF7D3FA00283DD02C48E2
S3150800112C02F0FCF92C4802F0F9F92C4801F064FDA0
S3150800113C2B4802F0F3F900222A4B1A7002F0BEF97A
S3150800114CFFF7E6F84DE6284802F0E8F9022002F027
S3150800115CD7F904F50C7001F04FFD0022214B1A70DB
S3150800116C70BD224802F0DAF9032002F0C9F91B48CF
S3150800117C01F042FD00221B4B1A7070BD002588E752
S3150800118C1B4802F0CBF9062002F0BAF9134801F015
S3150800119C33FD0022134B1A7070BD154802F0BEF9C8
S315080011AC072002F0ADF90D4801F026FD00220D4B83
S315080011BC1A7070BD704700BF28070020840B0020EA
S315080011CCC0520008080D0020D05200080053000831
S315080011DCF4510008E8520008045300085809002086
S315080011EC1C530008800B0020785200089C520008FB
S315080011FCEC5100084278007840EA02207047C27821
S3150800120C837843EA0222437843EA0223007840EAC9
S3150800121C032070470170090A417070470170C1F3C9
S3150800122C07234370C1F307438370090EC1707047D7
S3150800123C13462AB10A78027001300131013BF9D103
S3150800124C704701700130013AFBD1704730B4451C28
S3150800125C037808781B1A013A04D04C1C28462146F8
S3150800126C002BF4D0184630BC704700E001300378E8
S3150800127C0BB18B42FAD11846704702394369023BC7
S3150800128C994204D24389806A03FB01007047002007
S3150800129C704770B506460D4601F11A00FFF7AAFF0E
S315080012AC04463378032B00D070BD05F11400FFF704
S315080012BCA1FF44EA0040F7E770B506460C4615460A
S315080012CC91B204F11A00FFF7A5FF3378032B00D06F
S315080012DC70BD290C04F11400FFF79CFFF8E7000019
S315080012EC2DE9F04180460F4601F11A00FFF782FFFF
S315080012FC58BB3D7805F03F05013D05EB450305EB6D
S3150800130C83050126002404E04FF6FF73984222D188
S3150800131C01340C2C0DD8144B185D3844FFF76AFFB2
S3150800132C002EF1D0FE2D13D828F8150006460135E7
S3150800133CEEE73B7813F0400F10D0FE2D11D80023A2
S3150800134C28F815300120BDE8F0810020BDE8F081B1
S3150800135C0020BDE8F0810020BDE8F0810120BDE841
S3150800136CF0810020BDE8F081C85300082DE9F84348
S3150800137C80460F4691464B730F23CB7200240C7391
S3150800138C214607F11A00FFF745FF09F1FF3606EB70
S3150800139C460306EB8306254602E001340C2C11D8CD
S315080013AC4FF6FF739D4202D038F8165001360C4B97
S315080013BC185D29463844FFF72DFF002DEDD14FF661
S315080013CCFF75EAE74FF6FF739D4202D038F81630E0
S315080013DC0BB949F0400987F80090BDE8F88300BFBF
S315080013ECC853000870B582B0054616461C460B2233
S315080013FCFFF71EFF052C11D807231FE001310F2913
S3150800140C0DD802F0010000EB4303520813F4803F99
S3150800141CF4D083F4883383F02103EFE7234632882C
S3150800142C12B102360021EAE71C46E5E75A1E02A865
S3150800143C034403F8081C240909D0134604F00F02C8
S3150800144C02F130013929F1D902F13701EEE77E2193
S3150800145C0346134403F8081C00E00134944208D2EE
S3150800146C2B5D202BF9D104E0202018700C46072997
S3150800147C09D8611C2B19072AF6D802A8104410F8AB
S3150800148C080C0132F1E702B070BD01460B220020B0
S3150800149CC30143EA5003DBB208780344D8B20131DE
S315080014AC013AF5D17047016809B10A4603E04FF0D5
S315080014BCFF3308E0013213781F2B01D93A2BF9D1E7
S315080014CC3A2B02D000231846704710B44C1C0B78E4
S315080014DC303B092B07D8A24208D153B90132026016
S315080014EC184610BC70474FF0FF33F9E74FF0FF333F
S315080014FCF6E74FF0FF33F3E738B50C4620B105464F
S3150800150C03680BB11A781AB900232360092038BD71
S3150800151CD98882889142F7D1587803F033FA10F0BB
S3150800152C010FF1D12B682360002038BDF8B5C378BC
S3150800153C0BB90020F8BD0446C66A00F13007012332
S3150800154C32463946407803F06DFAA8B90023E370A1
S3150800155C236AF31AA269934210D2A57808E0A36904
S3150800156C1E44012332463946607803F05BFA013D86
S3150800157C012DF4D80020F8BD0120F8BD0020F8BDD7
S3150800158C70B5C36A8B4214D004460D46FFF7CEFFDE
S3150800159C064608B1304670BD01232A4604F13001CF
S315080015AC607803F0F9F910B101264FF0FF35E562C2
S315080015BCF0E70026EEE7000010B504460023C370DA
S315080015CC4FF0FF33C362FFF7DBFF08B1042010BDF1
S315080015DC04F22E20FFF70EFE4AF65523984201D048
S315080015EC032010BD04F16600FFF709FE20F07F40CA
S315080015FC084B98420CD004F18200FFF700FE20F04D
S3150800160C7F40044B984201D0022010BD002010BD2B
S3150800161C002010BD464154002DE9F04784B00E4613
S3150800162C174600230B60FFF73EFF051EC0F23581F7
S3150800163CA84B53F82540002C00F03381346007F092
S3150800164CFE0723787BB1607803F09CF910F0010F44
S3150800165C09D1002F00F0278110F0040F01D00A20C1
S3150800166C1CE100201AE100232370E8B2607003F035
S3150800167CE1F810F0010F01D003200FE127B110F0AB
S3150800168C040F01D00A2009E100212046FFF794FF38
S3150800169C02281DD00026042800F0078101282DD920
S315080016AC0D20FBE0002004AB03EB850343F8100C7C
S315080016BC0135032D0ED804F130002B0103F5DF7329
S315080016CC18440379002BEDD00830FFF798FDEAE7AC
S315080016DC0025EEE7002508E031462046FFF76CFFAB
S315080016EC0128D8D90135032DD5D804AB03EB8503CE
S315080016FC53F8106C002EEFD10320F1E704F13B00F0
S3150800170CFFF778FDB0F5007F01D00D20C6E004F197
S3150800171C4600FFF76FFD804620B904F15400FFF729
S3150800172C6EFD8046C4F8188094F8409084F80290B0
S3150800173C09F1FF33DBB2012B01D90D20AEE009FB11
S3150800174C08F994F83D706781002F00F0B0807B1E75
S3150800175C1F4201D00D20A1E004F14100FFF74AFD1C
S3150800176C8246208110F00F0F40F0A38004F143004D
S3150800177CFFF740FD054620B904F15000FFF73FFD81
S3150800178C054604F13E00FFF735FD0246002800F039
S3150800179C928009EB000303EB1A139D42C0F08D806F
S315080017ACED1AB5FBF7F5002D00F0898040F6F571BA
S315080017BC8D4260D801274FF6F5718D4200D9032763
S315080017CC02356561E661324422623344A362032F13
S315080017DC53D104F15A00FFF70DFD002871D1BAF167
S315080017EC000F70D104F15C00FFF709FD6062AD00D3
S315080017FC05F2FF15B8EB552F69D34FF0FF3323616C
S3150800180CE36080232371032F2CD104F16000FFF7CA
S3150800181CF1FC012826D1711C2046FFF7B1FE08BB46
S3150800182C0023237104F22E20FFF7E4FC4AF6552315
S3150800183C984217D104F13000FFF7E1FC264B984289
S3150800184C10D104F50570FFF7DAFC244B984209D140
S3150800185C04F50670FFF7D3FC206104F50770FFF753
S3150800186CCEFCE06027701E4A138801339BB21380A6
S3150800187CE380002012E002279DE7BAF1000F24D07E
S3150800188C4A446262022F01D16D00B1E705EB4503AC
S3150800189C05F0010505EB5305AAE70B2004B0BDE8D6
S315080018ACF0870C20FAE70020F8E70120F6E70D2070
S315080018BCF4E70D20F2E70D20F0E70D20EEE70D20FA
S315080018CCECE70D20EAE70D20E8E70D20E6E70D200A
S315080018DCE4E700BF480D0020525261417272416123
S315080018EC4C0D0020F8B5066801295DD97369994233
S315080018FC5CD20C463378022B30D0032B40D0012B0C
S3150800190C01D00120F8BD01EB5105316A01EB5521D7
S3150800191C3046FFF735FE10B14FF0FF30F8BD6F1C9F
S3150800192CC5F30805354495F83050316A01EB572153
S3150800193C3046FFF725FE10B14FF0FF30F8BDC7F360
S3150800194C08073E4496F8300045EA002014F0010FCB
S3150800195C01D00009F8BDC0F30B00F8BD316A01EBE4
S3150800196C14213046FFF70CFE10B14FF0FF30F8BDCE
S3150800197C600000F4FF7030303044FFF73BFCF8BDD4
S3150800198C316A01EBD4113046FFF7FAFD10B14FF06E
S3150800199CFF30F8BDA00000F4FE7030303044FFF77D
S315080019AC2EFC20F07040F8BD0120F8BD0120F8BDD2
S315080019BC2DE9F0410768B1F5001F02D30220BDE8F6
S315080019CCF08106460C4611F01F0F02D00220BDE826
S315080019DCF081316185681DB93B78022B00D97D6A87
S315080019EC75B93B89B3EB541F02D80220BDE8F081C8
S315080019FC7B6AB3617561B3690BBB0220BDE8F081E4
S31508001A0CB7F80A804FEA482801E0A4EB08044445D5
S31508001A1C0FD329463046FFF765FF0546B0F1FF3F61
S31508001A2C18D0012819D97B699842EED30220BDE853
S31508001A3CF08129463846FFF720FCB061DAE703EB5C
S31508001A4C5423B3613037C4F308043C44F4610020D2
S31508001A5CBDE8F0810120BDE8F0810220BDE8F081E7
S31508001A6C2DE9F84301297ED94369994201D3022607
S31508001A7C7AE017460C4605460378022B47D0032B0B
S31508001A8C57D0012B01D002266EE001EB5108016AF2
S31508001A9C01EB5821FFF774FD0646002864D108F1BE
S31508001AAC0109C8F3080814F0010423D005EB080350
S31508001ABC93F9303003F00F033A0102F47F621343B3
S31508001ACCDBB2A84488F830300123EB70296A01EBA5
S31508001ADC59212846FFF754FD0646002844D1C9F378
S31508001AEC08094CB1C7F30712A94489F83020012319
S31508001AFCEB7039E0FBB2E4E705EB090393F9302008
S31508001B0C22F00F02C7F303273A43D2B2ECE7016A75
S31508001B1C01EB1421FFF734FD064628BB600000F4E0
S31508001B2CFF703030B9B22844FFF774FB0123EB7011
S31508001B3C1AE0016A01EBD411FFF722FD064698B9A3
S31508001B4C27F07047A40004F4FE7430342C44204665
S31508001B5CFFF755FB00F0704139432046FFF75EFB53
S31508001B6C0123EB7000E002263046BDE8F8832DE928
S31508001B7CF04107460668884631B9F5688DB1736930
S31508001B8C9D420FD301250DE0FFF7ACFE0346012855
S31508001B9C47D9B0F1FF3F49D07269904246D34546C2
S31508001BAC00E001252C460CE021463846FFF79AFE44
S31508001BBC034670B1012839D0B0F1FF3F36D0AC429C
S31508001BCC33D0013473699C42EED3012D2BD90224F0
S31508001BDCEAE74FF0FF3221463046FFF741FF03464E
S31508001BEC10B9B8F1000F0ED1A3B9F4603369726954
S31508001BFC023A934201D2013B3361337943F0010334
S31508001C0C3371234612E0224641463046FFF728FF39
S31508001C1C0346E9E7012B01D0012307E04FF0FF3318
S31508001C2C04E0012302E0002300E000231846BDE887
S31508001C3CF081F8B50E460468012930D907461146D5
S31508001C4C63699E4201D302222AE05AB14FF0FF3251
S31508001C5C2046FFF705FF024620B121E063692E46B0
S31508001C6C9D421DD231463846FFF73CFE0546C8B1A3
S31508001C7C012819D0B0F1FF3F18D000223146204672
S31508001C8CFFF7EEFE024658B92369B3F1FF3FE5D0DC
S31508001C9C01332361237943F001032371DEE7022222
S31508001CAC1046F8BD0022FBE70222F9E70122F7E706
S31508001CBC2DE9F8430668036903F12005836913B90E
S31508001CCC0420BDE8F883B5F5001F02D30420BDE84F
S31508001CDCF88388460446C5F308078FB90133836130
S31508001CEC416941B93389B3EB551F09D80023836180
S31508001CFC0420BDE8F8837389013B13EA552307D002
S31508001D0C256107F130084644E6610020BDE8F883F2
S31508001D1CFFF7E8FD8146012848D9B0F1FF3F48D0C6
S31508001D2C736998423AD3B8F1000F04D10023A36122
S31508001D3C0420BDE8F88361692046FFF718FF814641
S31508001D4C10B90720BDE8F883012835D0B0F1FF3F5C
S31508001D5C35D03046FFF7EAFBA0BB4FF400720021E2
S31508001D6C06F13000FFF76DFA49463046FFF785FA5B
S31508001D7CF0624FF00008738998450BD20123F37073
S31508001D8C3046FFF7D3FB00BB08F10108F36A0133B1
S31508001D9CF362F0E7F36AA3EB0803F362C4F8149052
S31508001DAC49463046FFF769FAA061A9E70220BDE863
S31508001DBCF8830120BDE8F8830220BDE8F8830120EA
S31508001DCCBDE8F8830120BDE8F8830120BDE8F88357
S31508001DDCF8B504460F4606680021FFF7E9FD0246EA
S31508001DECC0B9002508E00135BD4213D001212046B3
S31508001DFCFFF75EFF024668B9A1693046FFF7C0FBDC
S31508001E0C024638B9E3691B78E52BECD0002BEAD0EF
S31508001E1C0025EBE7042A01D01046F8BD0722FBE79C
S31508001E2C2DE9F8430446884607684FF0FF094E46E5
S31508001E3C04252EE00F2B19D112F0400F06D091F87D
S31508001E4C0D9002F0BF02236963621646B24201D0B6
S31508001E5CFF2618E04B7B994501D0FF2613E0A06AB4
S31508001E6CFFF73EFA88B3013EF6B20CE026B90846EF
S31508001E7CFFF70BFB81452BD04FF0FF33636227E04E
S31508001E8CFF2600E0FF2600212046FFF711FF054636
S31508001E9CF0B9A169E1B13846FFF772FB0546B8B946
S31508001EACE1690A789AB1CB7A03F03F03A371E52A64
S31508001EBCE6D02E2AE6D023F02000082814BF0020EE
S31508001ECC01204045B6D0FF26DDE7FF26DBE70425D3
S31508001EDC0DB10023A3612846BDE8F88370B5044606
S31508001EEC05680669416AB1F1FF3F1CD0FFF760FD32
S31508001EFC0346B3B9A1692846FFF742FB034670B9F6
S31508001F0CE269E52111700122EA702269964206D926
S31508001F1C00212046FFF7CCFE03460028EAD0042B06
S31508001F2C03D0184670BD0023E3E70223F9E7000047
S31508001F3C2DE9F04F83B006468A46D1F80090856A9B
S31508001F4C002412E0013709EB070219F807302F2B8A
S31508001F5CF8D05C2BF6D0CAF800201F2822D84FF0F0
S31508001F6C040823E025F814803C46671C19F804007D
S31508001F7C1F28E8D92F28E6D05C28E4D0FE2C00F2DE
S31508001F8CDD80012100F0E2FF8046002800F0D880B1
S31508001F9C7F28E7D801466B48FFF767F90028E1D098
S31508001FAC062012E04FF0000800E0013C44B104F1B1
S31508001FBC0043013B35F81330202BF6D02E2BF4D0EA
S31508001FCC002325F814301CB9062003B0BDE8F08FA1
S31508001FDC0B222021306AFFF734F9002300E0013385
S31508001FEC35F81320202AFAD02E2AF8D01BB148F03F
S31508001FFC030800E0013C6CB104F10042013A35F8E3
S3150800200C12202E2AF6D14FF0080B4FF0000ACDF805
S3150800201C04A00AE0A2464FF0080B0022019204E045
S3150800202C4C450BD048F003084B4603F1010935F82B
S3150800203C137057B3202FF5D02E2FF1D0DA450FD2C7
S3150800204C4C450DD07F2F3FD8002F4AD148F00308B6
S3150800205C5F27336A03F80A704B460AF1010AE4E76C
S3150800206CBBF10B0F0FD04C4501D048F003084C457B
S3150800207C0BD3019B9B00DBB2019323464FF00B0B52
S3150800208C4FF0080AD1E748F00308336A1A78E52AAC
S3150800209C43D0BBF1080F43D0019901F00C020C2A6E
S315080020AC43D001F00303032B3FD018F0020F06D1DF
S315080020BC019B03F00303012B3AD0042A3BD0336A65
S315080020CC83F80B80002080E70021384600F03EFF9D
S315080020DC074618B1A0F180071B4BDF5D48F00208D4
S315080020ECB2E739461948FFF7C0F80028AED1A7F170
S315080020FC41039BB2192B04D8019B43F002030193AD
S3150800210CA7E7A7F161039BB2192BA2D8019B43F051
S3150800211C01030193203FBFB29BE705221A70B8E76B
S3150800212C019B9B00DBB20193B6E748F00208BCE7BB
S3150800213C48F01008C1E748F00808C0E7062044E74D
S3150800214C062042E7D853000848530008E453000811
S3150800215CF8B500238B758369002B6BD00D460646A4
S3150800216C436AB3F1FF3F13D0836A00249F1C188877
S3150800217C58B1002100F0EAFE30B1FE2C0CD82A1911
S3150800218C90753B460134F1E700242C440023A375D3
S3150800219CAC7D0022134612E00024F6E7E52317E08F
S315080021AC14B9A8182E278775A8182E274772013236
S315080021BC10E010271CE0A818837501320B460A2B71
S315080021CC1BD8F069591CC35C202BF7D0052BE5D01E
S315080021DC0929E5D0A8184372002CEED1A3F14100C9
S315080021ECC0B21928E7D8F069007B0829E1D8082776
S315080021FC0742E0D02033DBB2DDE734B9AB18002157
S3150800220C9975F3691B7B03B90A462A440023537252
S3150800221CF369DB7A2B72F0691C30FEF7F0FF286045
S3150800222CF0691830FEF7E6FFA880F0691630FEF75D
S3150800223CE1FFE880F8BD00002DE9F04781468846A5
S3150800224C01F11A00FEF7D6FFB0BB98F8005005F05E
S3150800225C3F05013D05EB450305EB830501270024E6
S3150800226C04E04FF6FF7398422FD101340C2C17D883
S3150800227C1C4B185D4044FEF7BDFF0646002FF0D0F8
S3150800228CFE2D1CD800F07EFE074605F1010A39F82A
S3150800229C150000F077FE874214D137465546E4E719
S315080022AC98F8003013F0400F12D0A7B139F8153052
S315080022BCA3B90120BDE8F0870020BDE8F08700200F
S315080022CCBDE8F0870020BDE8F0870020BDE8F08760
S315080022DC0120BDE8F0870120BDE8F0870020BDE8A5
S315080022ECF08700BFC85300082DE9F8430446D0F818
S315080022FC00800021FFF75CFB064600285ED14FF0F4
S3150800230CFF3363624FF0FF094F460AE04FF0FF3385
S3150800231C6362FF2700212046FFF7CAFC0646002801
S3150800232C4CD1A1694046FFF72BF90646002845D142
S3150800233CE5692B78002B40D0E97A01F03F02A271AF
S3150800234CE52BE3D011F0080F01D00F2ADED10F2AA6
S3150800235C14D027B92846FFF798F881452ED0216A5C
S3150800236CCB7A13F0010F04D10B222846FEF76EFF29
S3150800237C20B34FF0FF336362FF27CBE7A06A002830
S3150800238CC8D013F0400F06D095F80D9003F0BF0394
S3150800239C226962621F46BB4201D0FF27BAE76B7BF4
S315080023AC994501D0FF27B5E72946FFF745FF10B138
S315080023BC013FFFB2AEE7FF27ACE704263046BDE87F
S315080023CCF88330B583B004460191056801E0013302
S315080023DC0193019B1A782F2AF9D05C2AF7D0002290
S315080023ECA2601B781F2B1DD901A92046FFF7A0FD5B
S315080023FC0346F8B92046FFF777FF236ADA7A0346CD
S3150800240CD8B912F0040F15D1A37913F0100F1BD0FD
S3150800241C2169C1F30801303129442846FEF739FFF2
S3150800242CA060E1E7236A8022DA7200212046FFF7D2
S3150800243CBFFA0346184603B030BD0428FAD112F089
S3150800244C040FF7D10523F5E70523F3E72DE9F04744
S3150800245C84B00668D0F820A0D0F828809AF80B30FB
S3150800246C13F0A00F05D04FF00609484604B0BDE896
S3150800247CF087002400E0013438F81430002BFAD128
S3150800248C05460C22514601A8FEF7D2FE9DF80F30E0
S3150800249C13F0010F1ED000238AF80B30AB6201270C
S315080024AC632F0CD83B46424601A95046FEF79AFFC5
S315080024BC2846FFF719FF814608B90137F0E7642F5C
S315080024CC60D0B9F1040FD0D19DF80F308AF80B30D3
S315080024DCC5F828809DF80F3013F0020F2AD00C345B
S315080024EC2A4BA3FB0434A408013421462846FFF7DB
S315080024FC6FFC814608B9013C1ED1B9F1000FB4D165
S3150800250CA9693046FFF73CF881460028ADD1202250
S3150800251C0021E869FEF795FE0B22296AE869FEF7A1
S3150800252C87FEEA692B6ADB7A03F018031373012317
S3150800253CF3709AE70124D8E72969A1EB44112846D8
S3150800254CFFF736FA81460028D7D1286AFEF79DFF91
S3150800255C0746A9693046FFF713F881460028CCD1FF
S3150800256C3B46E2B2E969A86AFEF700FF0123F3705D
S3150800257C00212846FFF79CFB81460028BDD1013C6B
S3150800258CE7D1BAE74FF007096FE700BF4FECC44E27
S3150800259C70B50446FEF7CAFF054648B92378032BDF
S315080025AC08D000221146607802F094FA00B1012591
S315080025BC284670BD2379012BF3D104F130064FF46C
S315080025CC007200213046FEF73CFE4AF6552104F20D
S315080025DC2E20FEF71FFE0F493046FEF71FFE0E494A
S315080025EC04F50570FEF71AFE216904F50670FEF768
S315080025FC15FEE16804F50770FEF710FEE269013274
S3150800260CE26201233146607802F00CFA002323714A
S3150800261CC7E700BF525261417272416110B584B06E
S3150800262C01900091144604A840F8041DFEF73BFFE0
S3150800263C002818DB0E4B53F820300BB100221A7009
S3150800264C019B0BB100221A70019B094A42F82030F3
S3150800265C63B1012C01D0002006E0002201A96846CE
S3150800266CFEF7DAFF00E00B2004B010BD0020FBE7F4
S3150800267C480D00202DE9F04393B00191002800F095
S3150800268CAE80044616460023036002F01F073A463E
S3150800269C06A901A8FEF7C0FF0546002840F0A08051
S315080026AC069B079303AB0F934F4B1193019907A8FE
S315080026BCFFF787FE054620B90F9B93F90B30002BC5
S315080026CC2FDB16F01C0F79D0002D31D0042D2AD013
S315080026DC47F0080715B917F0080F35D14DB917F09B
S315080026EC080F01D047F02007069BDB6A23620E9B76
S315080026FC6362002D74D1069EDDF83880414630465B
S3150800270CFEF7C7FDA06008F11C00FEF778FDE06037
S3150800271C002363746361E36127742660F388A380DE
S3150800272C5EE00625CDE707A8FFF790FE0546CFE73E
S3150800273C9DF8223013F0110F04D116F0040FC9D0EE
S3150800274C0825C7E70725C5E7284E31460E980E30EB
S3150800275CFEF764FD31460E981630FEF75FFD202213
S3150800276C0E9BDA72069EDDF8388041463046FEF737
S3150800277C90FD8146002241463046FEF79DFD00211C
S3150800278C0E981C30FEF74AFD0122069BDA70B9F149
S3150800279C000FA3D0069BDE6A0022494607A8FFF75E
S315080027AC48FA0546002899D131460698FEF7E8FE00
S315080027BC054609F1FF33069AD3608FE7002D8DD1B4
S315080027CC9DF8223013F0100F07D116F0020F85D0A2
S315080027DC13F0010F82D0072580E704257EE709252B
S315080027EC284613B0BDE8F083500D00200000614860
S315080027FC2DE9F04F85B004468846164699460023BF
S3150800280CC9F8003003A9FEF777FE074630B9677C8E
S3150800281C27B9237C13F0010F04D10727384605B0D6
S3150800282CBDE8F08FE36862699B1AB34253D21E4621
S3150800283C51E0A1692046FFF755F85EE00227677458
S3150800284CECE701276774E9E702276774E6E70127CF
S3150800285C6774E3E74FF4007204F1280108EB402093
S3150800286CFEF7E6FC74E0E269019B934219D0237CDF
S3150800287C13F0400F0BD0012304F12801687802F0FD
S3150800288CD1F8002867D1237C23F040032374012355
S3150800289C019A04F128010398407802F07DF8002883
S315080028AC5CD1019BE3616169C1F30801C1F500754F
S315080028BCAE4200D2354628312A4621444046FEF718
S315080028CCB7FCA84463692B446361D9F800302B44E0
S315080028DCC9F80030761B002EA0D06369C3F3080232
S315080028EC002AE0D1039AB2F80AA00AF1FF3A1AEACA
S315080028FC532A08D1002B9CD1A06801289ED9B0F187
S3150800290CFF3F9ED0A061039DA1692846FEF7B5FC42
S3150800291C002899D00AEB000301935FEA562BA2D044
S3150800292C0AEB0B036A89934201D9A2EB0A0B5B46A5
S3150800293C019A4146687802F02FF8002887D1237C43
S3150800294C13F0400F04D0E069019BC01A834581D867
S3150800295C4FEA4B25B5E7012767745FE701276774CC
S3150800296C5CE72DE9F04F85B004468846164699462D
S3150800297C0023C9F8003003A9FEF7BEFD074630B997
S3150800298C677C27B9237C13F0020F04D10727384636
S3150800299C05B0BDE8F08F6369F3425FD3DE435DE0B3
S315080029AC00212046FFF7E3F86CE0A1692046FFF703
S315080029BCDEF867E002276774E9E701276774E6E73C
S315080029CC0123E26904F128010398407802F02AF8F9
S315080029DC20B9237C23F04003237462E00127677433
S315080029ECD5E702276774D2E701276774CFE74FF458
S315080029FC007208EB412104F12800FEF719FC237C30
S31508002A0C23F0400323746EE0E3699B4503D06269A7
S31508002A1CE3689A4269D3C4F81CB06069C0F308002D
S31508002A2CC0F50075AE4200D2354628302A464146D6
S31508002A3C2044FEF7FDFB237C43F040032374A84493
S31508002A4C63692B446361E268934238BF1346E360BB
S31508002A5CD9F800302B44C9F80030761B002E51D01B
S31508002A6C6369C3F30802002AD7D1039AB2F80AA0FD
S31508002A7C0AF1FF3A1AEA532A0FD1002B95D1A0680E
S31508002A8C00288DD000283DD0012893D0B0F1FF3F07
S31508002A9C93D0A061A36803B9A060237C13F0400F00
S31508002AAC8ED1039B0193A1691846FEF7E6FB834674
S31508002ABC002896D0D344750AA6D00AEB0503019ACA
S31508002ACC5289934201D9A2EB0A052B465A4641462E
S31508002ADC0198407801F0A6FF002885D1E169A1EBA1
S31508002AEC0B018D4283D86D02A9E701235A4604F1DE
S31508002AFC28010198407801F04FFF00288BD0012758
S31508002B0C677444E7237C43F0200323743FE770B5CE
S31508002B1C82B004460E460A290DD06368002B08DBE2
S31508002B2C5D1C23441E733C2D09DC6560A3680133C8
S31508002B3CA36002B070BD0D21FFF7E9FFEDE701AB0D
S31508002B4C2A4604F10C012068FFF70BFF019B9D42F6
S31508002B5C02D04FF0FF35E8E70025E6E730B583B03D
S31508002B6C044601A9FEF7C8FC0346C8B9227C12F034
S31508002B7C200F15D012F0400F0CD00123E26904F196
S31508002B8C28010198407801F04DFF88BB237C23F07F
S31508002B9C40032374216A0198FEF7F2FC034610B130
S31508002BAC184603B030BD656AEB7A43F02003EB7226
S31508002BBCA26829462068FEF77FFBE16805F11C0030
S31508002BCCFEF72CFB0B4905F11600FEF727FB002137
S31508002BDC05F11200FEF71EFB0122019BDA70019823
S31508002BECFFF7D6FC0346227C22F020022274D7E794
S31508002BFC0123D5E70000614810B582B00446FFF7FB
S31508002C0CADFF034610B1184602B010BD01A9204607
S31508002C1CFEF772FC03460028F5D100222260F2E783
S31508002C2C2DE9F04182B004460E4601A9FEF764FC74
S31508002C3C0746002840F0A280677C002F40F09E8053
S31508002C4CE368B34204D2227C12F0020F00D11E466E
S31508002C5C636900226261002E65D0019AB2F80A8077
S31508002C6C4FEA482873B1721EB2FBF8F2013BB3FB6C
S31508002C7CF8F18A4206D3C8F1000213406361F61ACA
S31508002C8CA56902E0A56815B1A56135BB4CE0002124
S31508002C9C2046FEF76CFF0546012804D0B0F1FF3F2D
S31508002CAC04D0A060F0E70227677467E00127677411
S31508002CBC64E029462046FEF715FE0546B5F1FF3FAA
S31508002CCC28D0012D29D9019B5B699D4225D2A56186
S31508002CDC636943446361A6EB080646450BD9237C16
S31508002CEC13F0020FE5D029462046FEF740FF0546AD
S31508002CFC0028E3D14646636933446361C6F3080387
S31508002D0C002B3FD029460198FEF7B7FA40B902279F
S31508002D1C677433E00127677430E0022767742DE087
S31508002D2C00EB562500E000256369C3F30803E3B1FD
S31508002D3CE269954219D0237C13F0400F0BD001237E
S31508002D4C04F128010198407801F06CFEE0B9237C67
S31508002D5C23F04003237401232A4604F12801019821
S31508002D6C407801F019FE90B9E5616369E26893420F
S31508002D7C04D9E360237C43F020032374384602B05D
S31508002D8CBDE8F0810025CFE701276774F6E7012730
S31508002D9C6774F3E730B591B001900D46002205A98A
S31508002DAC01A8FEF739FC044610B1204611B030BD17
S31508002DBC02AB0D930B4B0F93019905A8FFF701FB7B
S31508002DCC04460028F1D10D9B93F90B30002B06DB3A
S31508002DDC002DEAD0294605A8FFF7BAF9E5E7062437
S31508002DECE3E700BF500D002070B59CB0019002229D
S31508002DFC05A901A8FEF710FC059B1193044610B112
S31508002E0C20461CB070BD02AB1993264B1B93019937
S31508002E1C11A8FFF7D6FA04460028F1D1199B93F9A5
S31508002E2C0B30002B23DB9DF84A3013F0010F20D111
S31508002E3C0CBB059E18993046FEF72BFA05469DF8ED
S31508002E4C4A3013F0100F17D006960890002106A8E2
S31508002E5CFEF7AEFD044678B9002106A8FEF7E0FF9A
S31508002E6C034600B90723042B06D01C4604E00624A7
S31508002E7CDEE70724DCE70025002CC1D111A8FFF7F3
S31508002E8C2DF8044600B935B9002CB9D10598FFF7C9
S31508002E9C7FFB0446B4E70022294611A8FEF7C9FEB3
S31508002EAC0446F1E7500D00202DE9F04182B080462A
S31508002EBC0E46174605460024731E9C4214DA6B46CA
S31508002ECC012201A93846FFF793FC009B012B0BD175
S31508002EDC9DF804300D2BEFD06A1C2B7001340A2B8D
S31508002EEC01D01546E8E7154600232B701CB1404661
S31508002EFC02B0BDE8F0810020FAE710B594B004469C
S31508002F0C019100230293039303E0013401A8FFF710
S31508002F1CFEFD21780029F8D1029A002A0CDB6B46B3
S31508002F2C04A90198FFF71DFD48B9009B029A9A421D
S31508002F3C08D1039814B010BD4FF0FF30FAE74FF0E4
S31508002F4CFF30F7E74FF0FF30F4E700007F2816D97B
S31508002F5C31B1FF2812D88038094B33F81000704766
S31508002F6C00237F2B07D8064A32F81320904202D04A
S31508002F7C01339BB2F5E78033D8B27047002070470F
S31508002F8CEC530008B0F5805F06D2224B1A881AB3A8
S31508002F9C904221D3F0B406E01F4BF7E72B461A886C
S31508002FACCAB1904217D31D1D5B88190ADBB29C184F
S31508002FBCA04204DB0029F1D105EB4303EFE708290E
S31508002FCC09D8DFE801F0050A101316191C1F220090
S31508002FDC861A35F81600F0BC7047821A02F00103FF
S31508002FECC01A80B2F7E7103880B2F4E7203880B2FE
S31508002FFCF1E7303880B2EEE71A3880B2EBE70830E2
S3150800300C80B2E8E7503880B2E5E7A0F5E35080B225
S3150800301CE1E700BFEC540008E05600080022014B1B
S3150800302C5A707047500F0020034BFE22DA70187145
S3150800303C0222A3F844207047500F002010B5054C07
S3150800304C00232370FFF7EAFFFF23E3700123A4F89C
S3150800305C443010BD500F0020064BFF22DA700022B8
S3150800306C1A71597859719A71DA711A720622A3F87B
S3150800307C44207047500F002008B50020FFF7D4FFF6
S3150800308C08BD0000074BFF22DA70074A9A64002233
S3150800309C1A715A719A710722C3F807200822A3F8E5
S315080030AC44207047500F00209C570008044BFF2201
S315080030BCDA7042689A640122A3F84420704700BF6C
S315080030CC500F002008B53120FFF7AEFF08BD0000F1
S315080030DC38B5084CFF23E370002525716571FDF79B
S315080030ECA1FCA071E571257265720723A4F844301A
S315080030FC38BD00BF500F002038B5FDF74DFDE8B1BF
S3150800310CFFF78CFF0F4C01252570FF23E370102366
S3150800311C237100236371FDF785FCA071FDF794FC00
S3150800312CE071FDF791FCC0F3072020726572A57259
S3150800313C0823A4F84430FDF7AFFA38BD1020FFF782
S3150800314C73FF38BD500F002038B505464478FDF797
S3150800315C69FC0138844210DC0A4C6A78A16C201D83
S3150800316CFDF7F6F8FF23E3706A78A36C1344A3649F
S3150800317C6B780133A4F8443038BD2220FFF754FF8E
S3150800318C38BD00BF500F002038B504464578FDF70A
S3150800319C49FC0138854211DC61680A4DA9646278DC
S315080031AC281DFDF7D5F8FF23EB706278AB6C13443A
S315080031BCAB6463780133A5F8443038BD2220FFF799
S315080031CC33FF38BD500F0020F8B5054617460024C6
S315080031DC06E015F8013B1C44E4B2FDF74FFC3146FA
S315080031EC4E1E0029F5D13C600120F8BD10B5084CDF
S315080031FCFF23E370E21D4168A06CFFF7E5FF207121
S3150800320C00236371A3710823A4F8443010BD00BFD2
S3150800321C500F002038B505460D4B9C6CFDF702FC8B
S3150800322C6A1C411E2046FDF73BFA60B1084CFF2389
S3150800323CE370FDF7F7FB0138A36C0344A364012381
S3150800324CA4F8443038BD3120FFF7EEFE38BD00BF78
S3150800325C500F002038B504464578FDF7E3FB0238D5
S3150800326C85420EDC114BFF22DA700122A3F84420AA
S3150800327C617851B9FDF724FA90B93120FFF7D4FEDD
S3150800328C38BD2220FFF7D0FE38BDA21C074B986C20
S3150800329CFDF706FA28B16178044A936C0B449364DB
S315080032AC38BD3120FFF7C0FE38BD00BF500F0020D7
S315080032BC08B54168074B986CFDF7F6F930B1054B24
S315080032CCFF22DA700122A3F8442008BD3120FFF74B
S315080032DCABFE08BD500F002008B5FDF719F8034BD7
S315080032ECFF22DA700122A3F8442008BD500F0020F3
S315080032FC08B589B2FDF77EFB08BD0000054B002218
S3150800330C1A709A6483F84320A3F844209A705A706A
S3150800331C704700BF500F0020034B1B780BB10120E0
S3150800332C70470020704700BF500F00200022024B48
S3150800333C83F84320704700BF500F002008B5037868
S3150800334CFF2B04D0354A1278012A14D008BDFFF792
S3150800335CD3FE324B93F84330012B5AD02F4BB3F98B
S3150800336C44100029F2DD1846012380F84330033057
S3150800337CFFF7BEFFEAE7C93B352B46D8DFE803F073
S3150800338C3345454245453F363C3945454545454512
S3150800339C45454545454545454545454545454545C3
S315080033AC45454545454545454545241E1B21454549
S315080033BC4527452A2D30FFF7C7FECAE7FFF7E4FE77
S315080033CCC7E7FFF773FEC4E7FFF710FFC1E7FFF780
S315080033DC59FEBEE7FFF750FEBBE7FFF73DFEB8E721
S315080033ECFFF72CFEB5E7FFF715FFB2E7FFF732FF3D
S315080033FCAFE7FFF76DFEACE7FFF75AFFA9E7FFF754
S3150800340C6BFFA6E7FFF75EFEA3E72020FFF70CFE8F
S3150800341C9FE71020FFF708FEA0E700BF500F00201B
S3150800342C08B5054B9B6813F0010F01D0002008BDA9
S3150800343C00F0D2F8012008BD0008014008B5642048
S3150800344C00F09AF808BD08B500F09CF808BD000015
S3150800345C00B5C7B04FF48C720021684601F02CFEFB
S3150800346C69460948FFF796FC40B9009B53B19DF88D
S3150800347C083013F0100F02D1012000E0002047B0ED
S3150800348C5DF804FB0020FAE7B457000800487047BB
S3150800349CB457000808B50748002380F828320A22D2
S315080034AC0549FFF7E7F818B90122024B83F82822D9
S315080034BC08BD00BF9C0F0020A457000810B50D4B83
S315080034CC93F82832012B10D0FDF72EF900F164047D
S315080034DC094B1B6813F0400F03D1FDF725F98442FD
S315080034ECF6D20648FFF780FC10BD0248FFF784FBAE
S315080034FCEAE700BF9C0F002000440040B4570008C0
S3150800350C08B5054B93F82832012B00D008BD0248A4
S3150800351CFFF772FBFAE700BF9C0F002038B505468B
S3150800352C134B93F82832012B0CD11149FFF7E5FC04
S3150800353C002807DA0E48002380F82832FFF75CFBD0
S3150800354C00E001352B788BB10A4A5360FDF7ECF88D
S3150800355C00F10A04074B1B6813F0800FF1D1FDF735
S3150800356C8DFAFDF7E1F88442F4D2EAE738BD00BFDC
S3150800357C9C0F002000440040014B1880704700BF88
S3150800358CC811002008B5FDF7CFF80F4B1B689842F9
S3150800359C10D30E4B1B7873B901220C4B1A704FF4CF
S315080035AC80520B4B5A61FDF7BFF80A4B1B8818441F
S315080035BC054B186008BD0022044B1A704FF4805254
S315080035CC034B1A61EFE700BFCC110020CA1100208B
S315080035DC00100140C81100204FF48052014B1A61AB
S315080035EC704700BF0010014010B5064B4FF0FF3274
S315080035FCDA6000241C61DA60DC6001F0C3FC20464A
S3150800360C10BD00BF0010024010B504460E4B1878CA
S3150800361C4FF47A73B3FBF0F30C4A1068B0FBF3F073
S3150800362C00F0E4FB68B90F2C01D9012010BD00226B
S3150800363C21464FF0FF3000F0A7FB054B1C6000201D
S3150800364C10BD012010BD00BF010000200C00002099
S3150800365C0400002008B5074A136843F010031360EA
S3150800366C032000F07FFB0020FFF7CEFF01F0EAFBFA
S3150800367C002008BD00200240F0B44B6901229A4094
S3150800368C0468D4F8003223F47C534D6A43EA0523C4
S3150800369C43F00103C4F800320568D5F81C42D3433D
S315080036AC1C40C5F81C42CC69C4B90568D5F80C424F
S315080036BC1C40C5F80C4206684C69CF688D8845EAEB
S315080036CC0745483446F8345004684E698F680D88A7
S315080036DC45EA0745483604EBC6046560CC69012CF7
S315080036EC1ED08C69002C35D10568D5F804421C40CF
S315080036FCC5F804420C69002C33D10468D4F814526A
S3150800370C2B40C4F814320B6A012B31D00268D2F85C
S3150800371C003223F00103C2F800320020F0BC7047D7
S3150800372C0568D5F80C421443C5F80C4206684C6972
S3150800373C0F688D8845EA0745483446F834500468BE
S3150800374C4E698F688D8945EA0745483604EBC604E9
S3150800375C6560C6E70568D5F804421443C5F8044203
S3150800376CC8E70468D4F814321343C4F81432CAE709
S3150800377C0368D3F81C120A43C3F81C22C6E7704721
S3150800378C002800F09C8038B5044690F83C3003B30A
S3150800379C022384F83C302268136823F00203136072
S315080037AC2268136843F001031360FCF7C5FF05464E
S315080037BC23685A6812F0010F10D1FCF7BDFF401BA5
S315080037CC0A28F5D9032084F83C00002384F83D30F8
S315080037DC38BD80F83D30FFF7D2FFD9E75A6812F0AA
S315080037EC010F5DD0A269012A43D00022E1690129A3
S315080037FC41D022F04002216A01293FD022F0200252
S3150800380C616A01293DD022F01002A16A01293BD038
S3150800381C22F00802E16A012939D022F0040219685B
S3150800382C21F0FC010A431A602168A368E268134375
S3150800383C22691343626913436268013A1343CB61E5
S3150800384C2268136823F001031360FCF775FF05461D
S3150800385C23685A6812F0010F1CD0FCF76DFF401B49
S3150800386C0A28F5D9032084F83C00002384F83D3057
S3150800387C38BD8022BAE742F04002BCE742F020028B
S3150800388CBEE742F01002C0E742F00802C2E742F077
S3150800389C0402C4E75B6813F0010F08D0002300E0AC
S315080038AC002333B9042384F83C30012038BD0123A6
S315080038BCF7E700202064012384F83C3038BD01204A
S315080038CC70470000F8B503689A6812F0806F08D143
S315080038DC9A6812F0006F04D19A6812F0805F00F0B3
S315080038ECEC8090F83D20012A00F0EC80012280F84B
S315080038FC3D2090F83C20D2B2322A14D0622A16D037
S3150800390C222A03D0122280F83C2002E0422280F8B8
S3150800391C3C209A6812F0806F0DD19A6812F0006FED
S3150800392C61D0012508E0522280F83C20F1E772228A
S3150800393C80F83C20EDE7002505F1180212019C5889
S3150800394C04F001049C50026B9368002B4DD1066859
S3150800395C05F118031B01F4581768D26842EA475256
S3150800396C2243F2500E460446026B136903F00F030A
S3150800397C1361036805F1180109010B445A6822F012
S3150800398C0F025A6003680B445A68006B00690243BD
S3150800399C5A602268206BC77D837D1B0443EA076344
S315080039AC477D43EA0723007D03432F013A44C2F8B7
S315080039BC88312268206B90F81BE0837E1B0443EA4F
S315080039CC0E6390F819E043EA0E23007E03433A444B
S315080039DCC2F88C312268535843F001035350FCF754
S315080039ECABFE07463BE00225A6E7076805F1180477
S315080039FC240157F804E0566843EAC603D268134311
S31508003A0C43EA0E033B51ADE726B1FCF795FEC01B06
S31508003A1C864224D2032384F83C303DB9236880229D
S31508003A2C9A60002384F83D300320F8BD012D04D09C
S31508003A3C23684FF400029A60F3E723684FF40042B8
S31508003A4C9A60EEE7012D14D023689A681E4B9343AF
S31508003A5C14BF01230023A3B1B6F1FF3FD4D1002D27
S31508003A6CF0D123689A68194B934314BF012300239A
S31508003A7CF1E723689A68164B934314BF0123002376
S31508003A8CE9E794F83C30DBB2522B0ED0722B10D0EF
S31508003A9C422B03D0012384F83C3002E0222384F81D
S31508003AAC3C30002084F83D00F8BD322384F83C30C5
S31508003ABCF7E7622384F83C30F3E7042380F83C30BC
S31508003ACC0120F8BD0220F8BD000001100100000419
S31508003ADC00010008F8B50D46B9B990F83C30DBB2D0
S31508003AEC222B00F02F8190F83C30DBB2422B00F0F1
S31508003AFC2B8190F83C30DBB2622B00F0278190F8D2
S31508003B0C3C30DBB2722B00F02381012D15D090F8D6
S31508003B1C3D30012B00F02481012380F83D30B5BBE4
S31508003B2C90F83C30DBB2322B29D0522B2BD0122BEF
S31508003B3C1CD0222380F83C301BE090F83C30DBB2DA
S31508003B4C322B00F0078190F83C30DBB2522B00F098
S31508003B5C038190F83C30DBB2622B00F0FF8090F8C2
S31508003B6C3C30DBB2722BD2D10220F8BD422380F84E
S31508003B7C3C3016460446FCF7DFFD074638E0622360
S31508003B8C80F83C30F5E7722380F83C30F1E790F882
S31508003B9C3C30DBB2222B0BD0422B0DD0122B03D090
S31508003BAC322380F83C30E4E7522380F83C30E0E7D7
S31508003BBC622380F83C30DCE7722380F83C30D8E787
S31508003BCC26B1FCF7B9FDC01B864211D2032084F836
S31508003BDC3C00002384F83D30F8BD23681B6913F0BC
S31508003BEC030F0CBF0123002363B1B6F1FF3FE7D1E6
S31508003BFC002DF2D12368DB6813F0030F0CBF0123E9
S31508003C0C0023F1E7002D67D1636B216805F11B02D0
S31508003C1C12018A5802F004029A60002A5ED12168C1
S31508003C2C05F11B0212018A58520D1A60216805F11A
S31508003C3C1B021201895801F00201D960216811444E
S31508003C4C496801F00F01196121680A445268C2F3E8
S31508003C5C0722DA611D6221682A011144D1F8B811CC
S31508003C6C197521681144D1F8B811090A59752168D2
S31508003C7C1144D1F8B811090C997521681144D1F879
S31508003C8CB811090ED97521681144D1F8BC111976E9
S31508003C9C21681144D1F8BC11090A597621681144D6
S31508003CACD1F8BC11090C997621680A44D2F8BC21C2
S31508003CBC120EDA76D5B923682022DA604DBB94F851
S31508003CCC3C30DBB2622B1CD0722B1ED0422B11D08F
S31508003CDC012384F83C3010E0A36B96E7216805F1C4
S31508003CEC1B0212018A58D2085A609FE723682022C1
S31508003CFC1A61E3E7122384F83C30002084F83D006F
S31508003D0CF8BD322384F83C30F7E7522384F83C306C
S31508003D1CF3E794F83C30DBB2622B0BD0722B0DD048
S31508003D2C522B03D0012384F83C30E6E7122384F89F
S31508003D3C3C30E2E7222384F83C30DEE7422384F861
S31508003D4C3C30DAE70220F8BD0220F8BD0220F8BDA7
S31508003D5C0220F8BD0220F8BD0220F8BD0220F8BDED
S31508003D6C0220F8BD074AD36823F4E0631B041B0C36
S31508003D7C000200F4E060184340F0BF6040F40030E5
S31508003D8CD060704700ED00E030B4164BDB68C3F327
S31508003D9C0223C3F10704042C28BF04241D1D062D79
S31508003DAC17D9033B012505FA04F4013C2140994037
S31508003DBC05FA03F3013B1340194300280BDB0901F1
S31508003DCCC9B200F1604000F5614080F8001330BCC0
S31508003DDC70470023E6E700F00F000901C9B2024B51
S31508003DEC1954F4E700ED00E014ED00E00138B0F1E9
S31508003DFC807F0AD2064B5860F021064A82F82310B7
S31508003E0C0020986007221A6070470120704700BF8F
S31508003E1C10E000E000ED00E00022044BDA61044AF1
S31508003E2C136943F00103136101807047D811002010
S31508003E3C002002401A4BDB6813F0100F27D0194AE2
S31508003E4CD36943F00203D3611023154AD26812F0E2
S31508003E5C040F06D01349CA6942F00102CA6143F03D
S31508003E6C04030F4AD26912F0010F09D00D49CA6929
S31508003E7C42F00402CA610A49CA6922F00102CA61FF
S31508003E8C40F20112934204D0054AD36070470023CE
S31508003E9CDBE7034AD36923F00103D361704700BFFC
S31508003EAC00200240D81100200A4B1B6913F0800F22
S31508003EBC0DD0084B084A5A6002F188325A601B69C1
S31508003ECC13F0800F01D001207047002070470020A6
S31508003EDC704700BF0020024023016745034A136957
S31508003EEC43F0800313610020704700BF0020024096
S31508003EFC38B50446FCF720FC0546174BDB6813F06F
S31508003F0C010F0AD0B4F1FF3FF7D00CB3FCF714FC41
S31508003F1C401B8442F1D2032038BD0F4BDB6813F0EB
S31508003F2C200F02D020220C4BDA600B4BDB6813F007
S31508003F3C100F09D1084BDB6913F0010F04D1064B9E
S31508003F4CDB6813F0040F05D0FFF774FF012038BDAA
S31508003F5C032038BD002038BD002002402DE9F84367
S31508003F6C234C247E012C03D102231846BDE8F88382
S31508003F7C1E4690460F46044601221D4B1A764CF2F5
S31508003F8C5030FFF7B5FF034670BB012C29D0022C25
S31508003F9C24D04FF0040900244C4525D22101C1F147
S31508003FAC2002A1F1200328FA01F106FA02F21143C4
S31508003FBC26FA03F3194389B207EB4400FFF72CFFE3
S31508003FCC4CF25030FFF794FF0A4B1D6925F001059A
S31508003FDC1D61034640B90134E4B2DDE74FF002092E
S31508003FECD9E74FF00109D6E70021014A1176BCE75B
S31508003FFCD8110020002002400022064BDA61064B3D
S3150800400C1A6942F004021A611A6942F040021A61EE
S3150800401C704700BFD8110020002002400022064B32
S3150800402CDA61064B1A6942F002021A6158611A697A
S3150800403C42F040021A617047D81100200020024055
S3150800404C264B1B7E012B46D070B50E460546012223
S3150800405C224B1A760368022B20D04CF25030FFF70D
S3150800406C47FF90BB4FF0FF333360AC680121EA6819
S3150800407CAB6803EB82239C4228D22046FFF7CEFF7F
S3150800408C4CF25030FFF734FF154A136923F002033C
S3150800409C13610146B8B904F58064E8E74CF2503070
S315080040ACFFF726FF08B1012110E00120FFF7A4FF56
S315080040BC4CF25030FFF71CFF0146094A136923F0EE
S315080040CC0403136102E0346000E001210022034B73
S315080040DC1A76084670BD022108467047D81100208A
S315080040EC00200240264B98420DD0264B984216D0FB
S315080040FC254B98421FD0254B984228D0244B9842E2
S3150800410C31D00020704703F58433DA6842F0040294
S3150800411CDA60DA6822F00402DA600120704703F5E7
S3150800412C8233DA6842F00802DA60DA6822F00802AA
S3150800413CDA600120704703F58033DA6842F0100222
S3150800414CDA60DA6822F01002DA600120704703F5AB
S3150800415C7C43DA6842F02002DA60DA6822F0200240
S3150800416CDA600120704703F57843DA6842F04002BA
S3150800417CDA60DA6822F04002DA600120704700BF84
S3150800418C00080140000C01400010014000140140D9
S3150800419C00180140F0B50D68C5F30F2595FAA5F280
S315080041ACB2FA82F233E0A2F108044FF00113A340ED
S315080041BC43F080634E681F0EC45993FAA3FEBEFAE9
S315080041CC8EFE4FEA8E0E4FF00F0C0CFA0EFE24EAFA
S315080041DC0E0493FAA3FEBEFA8EFE4FEA8E0E06FA6C
S315080041EC0EF63443C451C6681C0A26EA040E94FA21
S315080041FCA4F4B4FA84F40E6906FA04F44EEA040438
S3150800420CC4604C68012C0FD0092C0DD0013235FA3C
S3150800421C02F337D0012393401D42F7D0072AC2D8A0
S3150800422C40F201139340C5E7C45993FAA3F6B6FABC
S3150800423C86F6B6004FF0030E0EFA06F624EA060EBC
S3150800424C93FAA3F6B6FA86F6B6008C6804FA06F65E
S3150800425C46EA0E06C651CC6893FAA3FEBEFA8EFE43
S3150800426C4FEA8E0E4FF0040C0CFA0EFE26EA0E06DA
S3150800427C93FAA3F3B3FA83F39B0004FA03F33343D9
S3150800428CC351C3E70120F0BD034B5B68C3F30313AB
S3150800429C024AD35CD840704700100240D457000835
S315080042AC034B5B68C3F30223024AD35CD8407047BE
S315080042BC00100240E4570008034B5B68C3F3C223A3
S315080042CC024AD35CD840704700100240E4570008F5
S315080042DC0B4B5B6803F480337BB1094B586800F4CD
S315080042EC00300130074BB3FBF0F0054B5B68C3F3AA
S315080042FC8343023303FB00F070470348F5E700BF1E
S3150800430C0010024000127A0000093D0008B5054B62
S3150800431C5B6803F00C03082B02D1FFF7D9FF08BD25
S3150800432C014808BD0010024000127A0010B5044678
S3150800433CFFF7ECFF2060FFF7A7FF6060FFF7B0FF01
S3150800434CA0606068FFF7B8FFE06010BD036813F063
S3150800435C400F29D110B4026822F47F4222F0BF0222
S3150800436C0B684C6823438C682343CC6823430C693D
S3150800437C23434C6923438C692343CC6923430C6A36
S3150800438C234313430360436823F00403CA8A134385
S3150800439C43600B6AB3F5005F02D0012010BC70476E
S315080043AC8B8C03610120F9E700207047C36813F46E
S315080043BC005F01D00020704770B584B00D460446E6
S315080043CCC36823F4B05323F00C034A68C9680A433C
S315080043DC29690A431343C360AB68026922F4405245
S315080043EC134303616B69426922F4407213434361B8
S315080043FC6846FFF79BFF1C4B9C422AD01B4B9C42E2
S3150800440C29D01B4B9C4228D0002343B3296849B3B7
S3150800441C03EB830303EB83038900B3FBF1F1154E1E
S3150800442CA6FB01356D092A0190B2642202FB15120E
S3150800443C13013233A6FB0323C3F34F1303F0F00225
S3150800444C024492B203F00F0313449BB2A3600120FB
S3150800445C06E0039BD9E7029BD7E7029BD5E700202A
S3150800446C04B070BD0020FBE7003801400044004052
S3150800447C004800401F85EB51014B1860704700BF80
S3150800448C0C000020024A137843F00103137070479E
S3150800449C0800002010B50D4BD860FCF745F900F163
S315080044AC32040A4B9B6813F0010F07D1FCF7E6FAA6
S315080044BCFCF73AF98442F4D2012300E000231BB935
S315080044CC024BD868C0B210BD002010BD00380040A1
S315080044DC08B54FF48052034B1A61FF20FFF7DAFF39
S315080044EC08BD00BF000C014010B50446FF20FFF7BD
S315080044FCD1FF207010BD38B5FCF716F900F5FA7522
S3150800450CFF20FFF7C7FF0446FCF7B8FAFF2C03D0C9
S3150800451CFCF70AF98542F3D8FF2C14BF00200120BA
S3150800452C38BD000010B54FF48052074B5A61FF2076
S3150800453CFFF7B0FFFFF7DFFF10B10124204610BDCF
S3150800454C0446FFF7C5FFF9E7000C014070B50546B0
S3150800455C0C46FFF7D0FF034608B9184670BD20462F
S3150800456CFFF798FFFD2C1BD04FF400762C4614F859
S3150800457C020BFFF78FFF6878FFF78CFF2546023E84
S3150800458CF4D1FF20FFF786FFFF20FFF783FFFF20FC
S3150800459CFFF780FF00F01F00052803D00023DCE797
S315080045AC0123DAE70123D8E770B504460E4610F066
S315080045BC800F07D1FFF78CFFFFF7B4FF60B9FF2513
S315080045CC284670BD00F07F0400213720FFF7ECFF6A
S315080045DC05460128F4D8EDE744F04000FFF75AFFEA
S315080045EC300EFFF757FFC6F30740FFF753FFC6F326
S315080045FC0720FFF74FFFF0B2FFF74CFFACB10120D5
S3150800460C082C14D0FFF746FF0C2C12D00A24FF20D6
S3150800461CFFF740FF0546FCF731FA15F0800FCFD0AF
S3150800462C631E13F0FF04F2D1CAE79520E8E787204A
S3150800463CE8E7FF20FFF72EFFE8E7F8B505460E4634
S3150800464CFCF772F800F16407FF20FFF723FF044616
S3150800465CFCF714FAFF2C03D1FCF766F88742F3D85B
S3150800466CFE2C01D00020F8BD6C1C2846FFF73CFF39
S3150800467C20460235FFF738FFFCF700FA023EF3D165
S3150800468CFF20FFF707FFFF20FFF704FF0120F8BD07
S3150800469C30B587B0214C4FF480532361204B0193DE
S315080046AC01230293022303930025049501A92046AE
S315080046BCFFF770FD4FF40043236100E00135092D27
S315080046CC1DD8FCF731F800F16404164B9B6813F0FF
S315080046DC020F03D1FCF728F88442F6D2FF22114BBD
S315080046ECDA60FCF721F800F164040E4B9B6813F0B2
S315080046FC010FE3D1FCF718F88442F6D2DEE7084B33
S3150800470C019309230293032303930023049301A91A
S3150800471C0248FFF73FFD07B030BD00BF000C014053
S3150800472C800080040038004030B593B0294B9A6954
S3150800473C42F008029A619A6902F008020292029AF9
S3150800474CDA6942F48042DA61DB6903F48043019347
S3150800475C019B214B03930123049302230593002405
S3150800476C06941E4D03A92846FFF714FD4FF48053F3
S3150800477C2B611B4B0393092304930323059306947C
S3150800478C03A92846FFF706FD164B03930423049347
S3150800479C03A92846FFF7FEFC08944FF48273099385
S315080047AC0A940B940C944FF400730D9338230E93C0
S315080047BC0F941094072311930B4C08A92046FFF766
S315080047CCC5FD236843F040032360FFF761FF13B070
S315080047DC30BD00BF0010024010001004000C014050
S315080047ECA000A004400040040038004010B58AB070
S315080047FC0F4C236823F040032360002300934FF4E7
S3150800480C827201920293039304934FF400720592F9
S3150800481C08220692079308930723099369462046AC
S3150800482CFFF794FD236843F0400323600AB010BDDC
S3150800483C00380040002840F09C80F0B583B0044650
S3150800484C4D4B1B7813F0020F04D04B4B1878C0B2A3
S3150800485C03B0F0BDFFF768FF4FF48052474B5A611F
S3150800486C00210846FFF7A0FE0546012810D0444B48
S3150800487C1C60FFF72DFE002C78D03F4A137803F006
S3150800488CFE031370FFF7B2FF3B4B1878C0B2DFE795
S3150800489CFBF74AFF00F57A764FF4D5710820FFF737
S315080048AC83FE012830D00021A920FFF77DFE0128C0
S315080048BC3ED92F4641E0FF20FFF7ECFD02AB2B4417
S315080048CC03F8040C0135EDB2032DF4D99DF8063026
S315080048DC012BCCD19DF80730AA2BC8D1FBF724FFA6
S315080048EC864206D94FF08041A920FFF75DFE0028C5
S315080048FCF4D1FBF719FF8642B9D900213A20FFF704
S3150800490C53FE054658B1B2E72546DDE7FF20FFF70B
S3150800491CC1FD02AB2B4403F8040C0135EDB2032D93
S3150800492CF4D99DF8043013F0400F1DD00C249EE7E3
S3150800493C0227A92501E0FCF7A1F8FBF7F5FE86424C
S3150800494C05D900212846FFF72FFE0028F3D1FBF7DF
S3150800495CEBFE86428BD94FF400711020FFF724FE2C
S3150800496C002884D13C4682E7042480E7FFF78AFDB9
S3150800497C8AE70120704700BF08000020000C0140A0
S3150800498CD011002018B9034B1878C0B27047012013
S3150800499C704700BF0800002008B10420704738B5DE
S315080049AC0D461C460BB9042038BD1C4B1B7813F05E
S315080049BC010F01D0032038BD194B1B6813F0080FE3
S315080049CC00D15202012C1AD011461220FFF7ECFD29
S315080049DC78B94FF400712846FFF72FFE28B105F574
S315080049EC0075FCF74BF8013CF3D100210C20FFF7BE
S315080049FCDBFDFFF76DFD201C18BF012038BD1146E5
S31508004A0C1120FFF7D1FD0028F3D14FF40071284689
S31508004A1CFFF713FE0028ECD00024EAE70800002074
S31508004A2CD011002008B10420704770B50D46164603
S31508004A3C1C460BB9042070BD244B1B7813F0010FD0
S31508004A4C01D0032070BD214B1B7813F0040F01D045
S31508004A5C022070BD1E4B1B6813F0080F00D15602BE
S31508004A6C012C1DD013F0060F28D131461920FFF75B
S31508004A7C9BFD78B9FC212846FFF768FD28B105F59A
S31508004A8C0075FBF7FBFF013CF4D1FD210020FFF775
S31508004A9C5DFDC0B1FFF71CFD201C18BF012070BDC1
S31508004AAC31461820FFF780FD0028F3D1FE21284651
S31508004ABCFFF74CFD0028EDD00024EBE721469720A4
S31508004ACCFFF772FDD1E70124E4E700BF08000020D8
S31508004ADCD011002030B585B018B10424204605B095
S31508004AEC30BD934B1B7813F0010F01D00324F5E767
S31508004AFC14460E2900F20D81DFE811F00F0016009E
S31508004B0C0B015F000B010B010B010B010B010B01D8
S31508004B1CBB00C200D100DF00F300FFF703FD00283D
S31508004B2C40F0F9800124A8E000210920FFF73CFD9C
S31508004B3C08B10124A1E010216846FFF77EFD002884
S31508004B4C00F0EB809DF800309B09012B24D09DF8D2
S31508004B5C053003F00F039DF80A2003EBD2139DF8DA
S31508004B6C0920520002F006021344DBB20233DBB210
S31508004B7C9DF808109DF80720920002EB91129DF8FB
S31508004B8C0610890201F440610A440132093B02FA13
S31508004B9C03F32360002470E09DF809309DF8082083
S31508004BAC03EB02239DF80720120402F47C1213442B
S31508004BBC01339B02236000245FE05E4B1B6813F0F5
S31508004BCC040F21D000218D20FFF7EEFC08B101243B
S31508004BDC53E0FF20FFF75EFC10216846FFF72DFD1A
S31508004BEC80B9012449E0FF20FFF754FC013DEDB2E2
S31508004BFC002DF8D19DF80A301A091023934023602A
S31508004C0C00243AE03025F3E700210920FFF7CCFC15
S31508004C1C08B1012431E010216846FFF70EFD002883
S31508004C2C7DD0444B1B6813F0020F11D09DF80A3047
S31508004C3C5B0003F07E039DF80B2003EBD2130133C4
S31508004C4C9DF80D209209013A93402360002414E044
S31508004C5C9DF80A30C3F384029DF80B10CB0003F0C1
S31508004C6C180303EB5113013302FB033323600024AF
S31508004C7C03E0304B1B6813700024FFF729FC2DE763
S31508004C8C00210920FFF790FC08B10124F5E7102153
S31508004C9C2046FFF7D2FC002843D10124EDE700217A
S31508004CAC0A20FFF781FC08B10124E6E7102120460B
S31508004CBCFFF7C3FCB8BB0124DFE700213A20FFF756
S31508004CCC73FC054648B10124D7E7FF20FFF7E2FB42
S31508004CDC6055FBF7D3FE0135EDB2032DF5D900244B
S31508004CECCBE7144B1B6813F0040F01D10124C4E75E
S31508004CFC00218D20FFF758FC08B10124BDE7FF20E1
S31508004D0CFFF7C8FB40212046FFF797FC68B901243A
S31508004D1CB3E70424B1E70024AFE70124ADE7012487
S31508004D2CABE70024A9E70024A7E70024A5E700BF02
S31508004D3C08000020D01100200F4B1A6842F001021F
S31508004D4C1A6059680D4A0A405A601A6822F0847229
S31508004D5C22F480321A601A6822F480221A605A6881
S31508004D6C22F4FE025A604FF41F029A604FF000625A
S31508004D7C034B9A60704700BF001002400000FFF812
S31508004D8C00ED00E008B5244A136823F0070343F046
S31508004D9C02031360136803F00703022B03D069217F
S31508004DAC1E48FBF787FD1E4A136843F480331360CD
S31508004DBC1B4B1B6813F4003FFAD0194A536823F4AB
S31508004DCC7C1343F4E8135360136843F08073136041
S31508004DDC134B1B6813F0007FFAD0114B5A6822F05C
S31508004DECF0025A605A6822F4E06242F480625A6011
S31508004DFC5A6822F460525A605A6822F0030242F04A
S31508004E0C02025A60064B5B6803F00C03082BF9D1B7
S31508004E1C0448FFF731FB08BD00200240EC57000898
S31508004E2C0010024000A24A0408B5FEF713FCFFF76F
S31508004E3CA9FF08BD08B5FFF7F7FFFBF783FDFBF7DE
S31508004E4C91FDFCE72DE9F0418CB0484B9A6942F08C
S31508004E5C01029A619A6902F001020692069ADA69C7
S31508004E6C42F08052DA61DA6902F080520592059AAC
S31508004E7C9A6942F004029A619A6902F00402049251
S31508004E8C049A9A6942F008029A619A6902F0080231
S31508004E9C0392039A9A6942F010029A619A6902F08F
S31508004EAC10020292029ADA6942F40032DA61DA697D
S31508004EBC02F400320192019ADA6942F00072DA6160
S31508004ECCDB6903F000730093009B294B07930123BE
S31508004EDC08930223099300240A94264D07A9284609
S31508004EECFFF758F94FF480532B6140F201130793DF
S31508004EFC4FF00408CDF82080A5F5006507A92846CB
S31508004F0CFFF748F940F20443079309270897032645
S31508004F1C09960A9407A92846FFF73CF940F60803B0
S31508004F2C0793CDF8208007A92846FFF733F9124BCB
S31508004F3C07930823089305F5806507A92846FFF704
S31508004F4C29F90E4B0793089709960A9407A9284638
S31508004F5CFFF720F90A4B5A6822F4C0425A605A687D
S31508004F6C42F480425A600CB0BDE8F0810010024051
S31508004F7C1000100400100140010001040200020494
S31508004F8C0000014008B51348FFF7ACF81248FFF7C4
S31508004F9CA9F81248FFF7A6F8114BDA6922F0007245
S31508004FACDA61DA6922F40032DA619A6922F01002BF
S31508004FBC9A619A6922F008029A619A6922F00402A7
S31508004FCC9A61DA6922F08052DA619A6922F0010252
S31508004FDC9A6108BD00100140000C01400008014010
S31508004FEC00100240002103E00B4B5B584350043180
S31508004FFC0A480B4B42189A42F6D30A4A02E0002397
S3150800500C42F8043B084B9A42F9D3FFF795FE00F099
S3150800501C0FF8FFF70FFF70470C5900080000002027
S3150800502CE0010020E0010020F8110020FEE7000056
S3150800503C70B500250C4E0D4CA41BA410A54209D125
S3150800504C00F050F800250A4E0A4CA41BA410A542E1
S3150800505C05D170BD56F8253098470135EEE756F858
S3150800506C253098470135F2E7045900080459000819
S3150800507C0459000808590008044B054A1B681B6AA2
S3150800508C002B08BF1346D3F8EC0070477C010020B0
S3150800509C1000002082B001B901A942B14BB11378B6
S315080050AC0B601278101C18BF012002B0704710460E
S315080050BCFBE76FF00100F8E703460244934200D180
S315080050CC704703F8011BF9E749B1FF2A8BBF8A23FE
S315080050DC0A700360012088BF4FF0FF3070470846FE
S315080050EC70470000F8B500BFF8BC08BC9E46704770
S311080050FCF8B500BFF8BC08BC9E4670471B
S315080051082E2E2F2E2E2F2E2E2F2E2E2F536F7572B4
S3150800511863652F41524D434D335F53544D333246E1
S31508005128312F63616E2E6300050206020603070324
S315080051380803090309040A040B040C040C050D05E5
S315080051480E050F050F061006100710082E2E2F2E0F
S315080051582E2F2E2E2F2E2E2F536F757263652F41E5
S31508005168524D434D335F53544D333246312F756193
S3150800517872742E6300000000303A00002E2E2F2E7F
S315080051882E2F2E2E2F2E2E2F536F757263652F6690
S31508005198696C652E630000004669726D77617265F1
S315080051A820757064617465207265717565737420FD
S315080051B864657465637465640A0D00004F70656EEE
S315080051C8696E67206669726D776172652066696CB3
S315080051D86520666F722072656164696E672E2E2E69
S315080051E8000000004552524F520A0D004F4B0A0D57
S315080051F8000000005374617274696E6720746865EC
S315080052082070726F6772616D6D696E67207365715C
S3150800521875656E63650A0D0050617273696E67205D
S315080052286669726D776172652066696C6520746F48
S315080052382064657465637420657261736520626CA1
S315080052486F636B732E2E2E0045726173696E672025
S31508005258000000002062797465732066726F6D20FD
S315080052686D656D6F727920617420307800000000D2
S3150800527852656164696E67206C696E652066726F2F
S315080052886D2066696C652E2E2E4552524F520A0DB0
S3150800529800000000496E76616C696420636865637E
S315080052A86B73756D20666F756E642E2E2E45525279
S315080052B84F520A0D0000000050726F6772616D6DDB
S315080052C8696E67200000000020627974657320748F
S315080052D86F206D656D6F72792061742030780000D3
S315080052E857726974696E672070726F6772616D208C
S315080052F8636865636B73756D2E2E2E00436C6F732A
S31508005308696E67206669726D776172652066696C71
S31508005318650A0D004669726D776172652075706455
S31508005328617465207375636365737366756C6C79E8
S3150800533820636F6D706C657465640A0D0000000063
S31508005348809A45418E418F804545454949498E8F02
S315080053589092924F994F555559999A9B9C9D9E9F05
S3150800536841494F55A5A5A6A7A8A9AAABACADAEAF06
S31508005378B0B1B2B3B4B5B6B7B8B9BABBBCBDBEBF9F
S31508005388C0C1C2C3C4C5C6C7C8C9CACBCCCDCECF8F
S31508005398D0D1D2D3D4D5D6D7D8D9DADBDCDDDEDF7F
S315080053A8E0E1E2E3E4E5E6E7E8E9EAEBECEDEEEF6F
S315080053B8F0F1F2F3F4F5F6F7F8F9FAFBFCFDFEFF5F
S315080053C801030507090E10121416181C1E00000002
S315080053D8222A3A3C3E3F7C7F000000002B2C3B3DAE
S315080053E85B5D0000C700FC00E900E200E400E0009D
S315080053F8E500E700EA00EB00E800EF00EE00EC0045
S31508005408C400C500C900E600C600F400F600F200AC
S31508005418FB00F900FF00D600DC00A200A300A500E7
S31508005428A7209201E100ED00F300FA00F100D1008F
S31508005438AA00BA00BF001023AC00BD00BC00A1003A
S31508005448AB00BB00912592259325022524256125C5
S315080054586225562555256325512557255D255C253D
S315080054685B251025142534252C251C2500253C25C7
S315080054785E255F255A255425692566256025502504
S315080054886C256725682564256525592558255225D7
S3150800549853256B256A2518250C25882584258C25EA
S315080054A890258025B103DF009303C003A303C30334
S315080054B8B500C403A6039803A903B4031E22C603AA
S315080054C8B50329226122B1006522642220232123FB
S315080054D8F7004822B0001922B7001A227F20B20026
S315080054E8A025A00061001A03E0001703F8000703C7
S315080054F8FF00010078010001300132010601390177
S3150800550810014A012E017901060180014D00430266
S31508005518810182018201840184018601870187014C
S3150800552889018A018B018B018D018E018F019001FA
S315080055389101910193019401F60196019701980149
S3150800554898013D029B019C019D0120029F01A00133
S31508005558A001A201A201A401A401A601A701A7010D
S31508005568A901AA01AB01AC01AC01AE01AF01AF01BB
S31508005578B101B201B301B301B501B501B701B8016B
S31508005588B801BA01BB01BC01BC01BE01F701C001E3
S31508005598C101C201C301C401C501C401C701C801CB
S315080055A8C701CA01CB01CA01CD011001DD010100FD
S315080055B88E01DE011201F3010300F101F401F40181
S315080055C8F8012801220212013A020900652C3B0259
S315080055D83B023D02662C3F02400241024102460256
S315080055E80A015302400081018601550289018A0190
S315080055F858028F015A0290015C025D025E025F0240
S3150800560893016102620294016402650266026702F6
S31508005618970196016A02622C6C026D026E029C0161
S31508005628700271029D01730274029F017602770265
S31508005638780279027A027B027C02642C7E027F0257
S31508005648A60181028202A9018402850286028702CE
S31508005658AE014402B101B20145028D028E028F02E3
S3150800566890029102B7017B030300FD03FE03FF03C3
S31508005678AC0304008603880389038A03B10311036C
S31508005688C2030200A303A303C4030803CC0303004D
S315080056988C038E038F03D8031801F2030A00F90353
S315080056A8F303F403F503F603F703F703F903FA0319
S315080056B8FA033004200350041007600422018A0400
S315080056C83601C1040E01CF040100C004D004440108
S315080056D861052604000000007D1D0100632C001EDC
S315080056E89601A01E5A01001F0806101F0606201F4D
S315080056F80806301F0806401F0606511F0700591FCF
S31508005708521F5B1F541F5D1F561F5F1F601F080629
S31508005718701F0E00BA1FBB1FC81FC91FCA1FCB1F81
S31508005728DA1FDB1FF81FF91FEA1FEB1FFA1FFB1FFB
S31508005738801F0806901F0806A01F0806B01F040049
S31508005748B81FB91FB21FBC1FCC1F0100C31FD01F2B
S315080057580206E01F0206E51F0100EC1FF21F010002
S31508005768FC1F4E21010032217021100284210100FC
S315080057788321D0241A05302C2F04602C0201672CAB
S315080057880601752C0201802C6401002D260841FFAC
S315080057981A0300004F70656E424C54002F626F6FF3
S315080057A8746C6F672E747874000000002F64656D3A
S315080057B86F70726F675F6F6C696D65785F73746D0C
S315080057C83332703130332E7372656300000000007F
S315080057D8000000000102030406070809000000008B
S315080057E8010203042E2E2F6D61696E2E63000000D8
S315080057F84300504F534958002E00002020202020EF
S31508005808202020202828282828202020202020205A
S31508005818202020202020202020202088101010104A
S31508005828101010101010101010101004040404049E
S3150800583804040404041010101010101041414141CA
S3150800584841410101010101010101010101010101B2
S3150800585801010101010110101010101042424242C4
S315080058684242020202020202020202020202020282
S3150800587802020202020210101010200000000000A6
S315080058880000000000000000000000000000000002
S3150800589800000000000000000000000000000000F2
S315080058A800000000000000000000000000000000E2
S315080058B800000000000000000000000000000000D2
S315080058C800000000000000000000000000000000C2
S315080058D800000000000000000000000000000000B2
S315080058E800000000000000000000000000000000A2
S311080058F800000000000000000000000096
S309080059043101000857
S309080059080D01000877
S3150800590C04010000100000000100000000A24A0477
S3150800591C430000000000000000000000000000002A
S3150800592C000000000000000000000000000000005D
S3150800593C430000000000000000000000000000000A
S3150800594C000000000000000000000000000000003D
S3150800595C43000000000000000000000000000000EA
S3150800596C000000000000000000000000000000001D
S3150800597C43000000000000000000000000000000CA
S3150800598C00000000000000000000000000000000FD
S3150800599C43000000000000000000000000000000AA
S315080059AC00000000000000000000000000000000DD
S315080059BC430000000000000000000000000000008A
S315080059CC00000000000000000000000000000000BD
S315080059DC430000000000000000000000000000006A
S315080059EC000000000000000000000000000000009D
S315080059FCD5500008A1500008000000000258000805
S31508005A0C00580008015800080158000801580008F9
S31508005A1C01580008015800080158000801580008E8
S31508005A2C0158000801580008FFFFFFFFFFFFFFFFA2
S31508005A3CFFFFFFFFFFFF00000100415343494900E8
S31508005A4C000000000000000000000000000000003C
S31508005A5C00000000000000000000415343494900C3
S31508005A6C000000000000000000000000000000001C
S31508005A7C000000000000000000000000800100206B
S31508005A8C00000000000000000000000000000000FC
S31508005A9C00000000000000000000000000000000EC
S31508005AAC00000000000000000000000000000000DC
S31508005ABC00000000000000000000000000000000CC
S31508005ACC00000000000000000000000000000000BC
S31508005ADC00000000000000000000000000000000AC
S70508004FF1B2
